:020000040000fa
:08000000101b040000000000c9
:020000040000fa
:10000800041a0000081a00000c1a0000101a000058
:10001800141a00000c1b00000c1b00000c1b000035
:10002800181a00001c1a0000201a0000241a0000e8
:100038000c1b0000281a00002c1a0000301a0000bf
:10004800341a0000381a00003c1a0000401a000058
:10005800441a0000481a00000c1b00000c1b00008a
:100068004c1a0000501a0000541a0000581a0000d8
:100078005c1a00000c1b0000601a0000641a0000e3
:100088000c1b0000681a00006c1a0000701a0000af
:10009800741a0000781a00007c1a0000801a000008
:1000a800841a0000881a00000c1b00000c1b0000ba
:1000b8000c1b00008c1a0000901a0000941a000013
:1000c800981a00009c1a0000a01a0000a41a000048
:1000d800a81a0000ac1a00000c1b00000c1b000042
:1000e8000c1b0000b01a0000b41a00000c1b000022
:1000f8000c1b0000b81a0000bc1a00000c1b000002
:100108000c1b00000c1b00000c1b00000c1b00004b
:100118000c1b00000c1b0000c01a00000c1b000088
:100128000c1b0000c41a0000c81a0000cc1a0000fa
:100138000c1b00000c1b00000c1b00000c1b00001b
:10014800d01a00000c1b00000c1b00000c1b000048
:100158000c1b0000d41a00000c1b00000c1b000034
:100168000c1b0000d81a0000dc1a0000e01a00007e
:10017800e41a0000e81a0000ec1a0000f01a000067
:10018800f41a0000f81a0000fc1a0000001b000016
:10019800041b0000081b00000c1b00000c1b0000c7
:1001a8000c1b00000c1b00000c1b00000c1b0000ab
:1001b8000c1b00000c1b00000c1b00000c1b00009b
:1001c8000c1b00000c1b00000c1b00000c1b00008b
:1001d8000c1b00000c1b00000c1b00000c1b00007b
:1001e8000c1b00000c1b00000c1b00000c1b00006b
:0801f8000c1b00000c1b0000b1
:020000040000fa
:04020800ec1b0000eb
:020000040000fa
:04020c00ec1b0000e7
:020000040000fa
:04021000ec1b0000e3
:020000040000fa
:04021400ec1b0000df
:020000040000fa
:04021800ec1b0000db
:020000040000fa
:04021c00ec1b0000d7
:020000040000fa
:04022000ec1b0000d3
:020000040000fa
:04022400ec1b0000cf
:020000040000fa
:04022800ec1b0000cb
:020000040000fa
:04022c00ec1b0000c7
:020000040000fa
:04023000ec1b0000c3
:020000040000fa
:04023400ec1b0000bf
:020000040000fa
:04023800ec1b0000bb
:020000040000fa
:04023c00ec1b0000b7
:020000040000fa
:04024000ec1b0000b3
:020000040000fa
:04024400ec1b0000af
:020000040000fa
:04024800ec1b0000ab
:020000040000fa
:04024c00ec1b0000a7
:020000040000fa
:04025000ec1b0000a3
:020000040000fa
:04025400ec1b00009f
:020000040000fa
:04025800ec1b00009b
:020000040000fa
:04025c00ec1b000097
:020000040000fa
:04026000ec1b000093
:020000040000fa
:04026400ec1b00008f
:020000040000fa
:04026800ec1b00008b
:020000040000fa
:04026c00ec1b000087
:020000040000fa
:04027000ec1b000083
:020000040000fa
:04027400ec1b00007f
:020000040000fa
:04027800ec1b00007b
:020000040000fa
:04027c00ec1b000077
:020000040000fa
:04028000ec1b000073
:020000040000fa
:04028400ec1b00006f
:020000040000fa
:04028800ec1b00006b
:020000040000fa
:04028c00ec1b000067
:020000040000fa
:04029000ec1b000063
:020000040000fa
:04029400ec1b00005f
:020000040000fa
:04029800ec1b00005b
:020000040000fa
:04029c00ec1b000057
:020000040000fa
:0402a000ec1b000053
:020000040000fa
:0402a400ec1b00004f
:020000040000fa
:0402a800ec1b00004b
:020000040000fa
:0402ac00ec1b000047
:020000040000fa
:0402b000ec1b000043
:020000040000fa
:0402b400ec1b00003f
:020000040000fa
:0402b800ec1b00003b
:020000040000fa
:0402bc00ec1b000037
:020000040000fa
:0402c000ec1b000033
:020000040000fa
:0402c400ec1b00002f
:020000040000fa
:0402c800ec1b00002b
:020000040000fa
:0402cc00ec1b000027
:020000040000fa
:0402d000ec1b000023
:020000040000fa
:0402d400ec1b00001f
:020000040000fa
:0402d800ec1b00001b
:020000040000fa
:0402dc00ec1b000017
:020000040000fa
:0402e000ec1b000013
:020000040000fa
:0402e400ec1b00000f
:020000040000fa
:0402e800ec1b00000b
:020000040000fa
:0402ec00ec1b000007
:020000040000fa
:0402f000ec1b000003
:020000040000fa
:0402f400ec1b0000ff
:020000040000fa
:0402f800ec1b0000fb
:020000040000fa
:0402fc00ec1b0000f7
:020000040000fa
:04030000ec1b0000f2
:020000040000fa
:04030400ec1b0000ee
:020000040000fa
:04030800ec1b0000ea
:020000040000fa
:04030c00ec1b0000e6
:020000040000fa
:04031000ec1b0000e2
:020000040000fa
:04031400ec1b0000de
:020000040000fa
:04031800ec1b0000da
:020000040000fa
:04031c00ec1b0000d6
:020000040000fa
:04032000ec1b0000d2
:020000040000fa
:04032400ec1b0000ce
:020000040000fa
:04032800ec1b0000ca
:020000040000fa
:04032c00ec1b0000c6
:020000040000fa
:04033000ec1b0000c2
:020000040000fa
:04033400ec1b0000be
:020000040000fa
:04033800ec1b0000ba
:020000040000fa
:04033c00ec1b0000b6
:020000040000fa
:04034000ec1b0000b2
:020000040000fa
:04034400ec1b0000ae
:020000040000fa
:04034800ec1b0000aa
:020000040000fa
:04034c00ec1b0000a6
:020000040000fa
:04035000ec1b0000a2
:020000040000fa
:04035400ec1b00009e
:020000040000fa
:04035800ec1b00009a
:020000040000fa
:04035c00ec1b000096
:020000040000fa
:04036000ec1b000092
:020000040000fa
:04036400ec1b00008e
:020000040000fa
:04036800ec1b00008a
:020000040000fa
:04036c00ec1b000086
:020000040000fa
:04037000ec1b000082
:020000040000fa
:04037400ec1b00007e
:020000040000fa
:04037800ec1b00007a
:020000040000fa
:04037c00ec1b000076
:020000040000fa
:04038000ec1b000072
:020000040000fa
:04038400ec1b00006e
:020000040000fa
:04038800ec1b00006a
:020000040000fa
:04038c00ec1b000066
:020000040000fa
:04039000ec1b000062
:020000040000fa
:04039400ec1b00005e
:020000040000fa
:04039800ec1b00005a
:020000040000fa
:04039c00ec1b000056
:020000040000fa
:10340000101b040000000000ec1b04000000000082
:10341000ec1b040000000000ec1b04000000000096
:10342000ec1b040000000000ec1b04000000000086
:10343000ec1b040000000000ec1b04000000000076
:10344000ec1b040000000000d81b0400000000007a
:10345000ec1b040000000000ec1b04000000000056
:10346000ec1b040000000000ec1b04000000000046
:10347000ec1b040000000000ec1b04000000000036
:10348000ec1b040000000000ec1b04000000000026
:10349000ec1b040000000000ec1b04000000000016
:1034a000ec1b040000000000ec1b04000000000006
:1034b000ec1b040000000000ec1b040000000000f6
:1034c000ec1b040000000000ec1b040000000000e6
:1034d000ec1b040000000000ec1b040000000000d6
:1034e000ec1b040000000000ec1b040000000000c6
:1034f000ec1b040000000000ec1b040000000000b6
:10350000ec1b040000000000ec1b040000000000a5
:10351000ec1b040000000000ec1b04000000000095
:10352000ec1b040000000000ec1b04000000000085
:10353000ec1b040000000000ec1b04000000000075
:10354000ec1b040000000000ec1b04000000000065
:10355000ec1b040000000000ec1b04000000000055
:10356000ec1b040000000000ec1b04000000000045
:10357000ec1b040000000000ec1b04000000000035
:10358000ec1b040000000000ec1b04000000000025
:10359000ec1b040000000000ec1b04000000000015
:1035a000ec1b040000000000ec1b04000000000005
:1035b000ec1b040000000000ec1b040000000000f5
:1035c000ec1b040000000000ec1b040000000000e5
:1035d000ec1b040000000000ec1b040000000000d5
:1035e000ec1b040000000000ec1b040000000000c5
:1035f000ec1b040000000000ec1b040000000000b5
:10360000ec1b040000000000ec1b040000000000a4
:10361000ec1b040000000000ec1b04000000000094
:020000040000fa
:103620000fa320000e7f24000e0188000000000080
:10363000000020000000e000020032000001200035
:103640002002880014000700650007000000e00069
:1036500003003a00409d23000100200002003700d3
:103660000000200001002000810f700001003200e6
:1036700014000700000020000000e00002003200fb
:1036800000000200000000002036020000000000e0
:103690000040da000000fe004440a9004011200074
:1036a0000000e0000300320000002000a0018800bc
:1036b0004440a800000006008a1f78008b1f780095
:1036c0000000060091018800800478000000eb00f3
:1036d0001a003700e284440032a0b4009905ba0011
:1036e000e284440032a0b4009906ba00e2844400a7
:1036f00032a0b4000006eb00476fde00fd07b20009
:10370000636ce10003003a00ebff07000000eb00f0
:103710000a003700606ce10004003a00005deb0035
:103720008b05e900fdff3e00040037006168e10001
:10373000010032000086eb000b00070019c7ba0039
:103740001905ba000e04e00003003a000a00e00088
:10375000e0ff3a0000000600fe07b2009e0188006c
:103760008a047800f5ff3700395dba008b05e9005f
:103770000c003200295dba008b05e9000800320018
:103780000c00e00003003a00e284440032a0b400e0
:10379000f5ff370019ddba008b05e900faff3a00a2
:1037a0008904e800e184440032a0b400000006006f
:1037b0003400f800881f780008002000a801880065
:1037c0004f0478000000fa008460a9000080fa002d
:1037d0003400f900004006000040da000000fe005e
:1037e000000005008001780002003700b159780020
:1037f0000201e9000200e000fcff3a0000000600c0
:10380000889fbe008a9fbe00800478000200e0000e
:103810005b00320001407800814c780082814400d6
:10382000f1f99f00e20f51005500360091449800d5
:10383000a1449800e1f99f00d1f99f00e60f5100e3
:103840004f003600b1449800c1f99f00e80f5100c5
:103850004b0036000905ea00630565000a84440050
:103860000a055100c1ff2f00010565000080fb0023
:103870008000eb001210200013102000440007000d
:10388000008cbe000a01440060b99f0071b99f001e
:10389000e80f55003a0036002004980031049800e3
:1038a000400498005104980020b99f0031b99f004e
:1038b00040b99f0051b99f00f80f55003000360005
:1038c0006004980071049800000c9800110c980096
:1038d000200c9800310c9800400c9800510c980076
:1038e00020b19f0031b19f0040b19f0051b19f00b6
:1038f00060b19f0071b19f0000b99f0011b99f0096
:10390000640164007801410002044400020555008e
:103910006011b8000203be000002be000403be0036
:103920006022b80000007200818072000201730002
:103930008381730010003700009cbe000294be001b
:1039400040049800510498006204980073049800a1
:10395000000c9800110c9800220c9800330c980071
:10396000400c9800510c9800620c9800730c980061
:103970000a02b1000802b000ff0f5500eeff3e0042
:10398000090078004f05be004f04be00000006008d
:10399000020ab900001bb9000200b8008100420011
:0839a000810043000000060055
:020000040000fa
:1039a80012010000000200000200000000080000f0
:1039b800d80400000a000000000100000102000015
:1039c800000100000902000043000000020100009d
:1039d80000c00000320900000400000000010000df
:1039e8000202000001000000052400000010000091
:1039f8000104000024020000020500002406000063
:103a0800000100000524000001000000010700007b
:103a180005810000030a00000002000009040000fc
:103a280001000000020a000000000000000700007a
:103a38000502000002400000000000000705000029
:103a480082020000400000000000000004030000a3
:103a5800090400000a0300004d0000004f000000a8
:103a68004700000049000000260300005500000040
:103a78004d0000004f000000470000004900000012
:103a88003200000020000000530000006500000024
:103a98007200000069000000610000006c00000076
:103aa80020000000700000006f000000720000009d
:103ab80074000000e69c00002a9d00002e9d000076
:103ac800389d0000020400000e0100000f110000e4
:103ad8000f000000020400000e1100001f1000007b
:103ae8000e000000020400000c04000004040000a2
:103af8000e000000020400000e1100001111000069
:103b08000e00000002040000111100001113000053
:103b18000d0000000a000000111100001113000040
:103b28000d000000050a000011110000111300002b
:103b38000d000000050a00000e1100001111000020
:103b48000e000000754d00004f470000493200008c
:103b580020550000534200002d550000415200003e
:103b6800540a000000390000363000003020000000
:103b78006270000073200000384e00003120000001
:103b880020200000003100003135000032300000f4
:103b9800302000006270000073200000384e0000e2
:103ba80031200000000000003031000032330000f6
:103bb8003435000036370000383900004142000033
:083bc8004344000045460000e3
:020000040000fa
:103bd0000200fa009ec0a9000080eb00702488005b
:103be0000080eb0050248800aa24ef00420020004f
:103bf0008000eb00c04a200001ff070020002000e9
:103c000030258800a824ef008644a900f009200090
:103c100080248800f00920006024880082c4a80065
:103c20008804a80000a020004800de00c02488000e
:103c30000040eb00004f7800070037001e80fb00bb
:103c4000c200dd0000a02000008140006000b8003c
:103c50000089be001e4fe8001e407800eb4f500068
:103c6000f6ff36009424a8009624ef0094a4a9003f
:103c70009424a9008000200050248800a09b2000ec
:103c80008040eb0001487800009c20008040eb0061
:103c900001487800014e8000f00f20000080600095
:103ca000004e8800114e800000f02f000080600060
:103cb000104e880050248000680060000000e00082
:103cc000ecff3a0010c0b30013e8b70010c0b30017
:103cd00014e8b7001568ef001668ef000d68ef00f4
:103ce0000040eb00004f7800170037001e80fb00fb
:103cf00080004000209b2000008040008000eb00fe
:103d0000010878001e80fb0080004000c09a20005f
:103d1000008040008000eb00010878009e80fb00de
:103d2000609c2000008040008040eb00014878004b
:103d30009e80fb00a09c2000008040008040eb00a3
:103d4000014878001e4fe8001e407800e24f500006
:103d5000e6ff360080a02000904d8800d0002000b3
:103d600050258800d09c20001050880000a0200022
:103d700081c0b3000148780010a0200041c0b3000a
:103d80000148780010a020001040780080407800a2
:103d90000174a00010a02000014878000268ef0024
:103da0001828ef001a28ef001c68ef000028ef0029
:103db0000080fa00000006000200fa0000408000c7
:103dc0000000e00013003a009424ef008c24ef0080
:103dd0002000200030258800a824ef008644a90098
:103de000f009200080248800f00920006024880069
:103df00082c4a800010037009404a800a024800019
:103e0000610060000000e000fbff320010002000b5
:103e10000040880000408000e10f50000c003a0094
:103e2000a124800000042000008060000000e00069
:103e300007003a000080eb00502488008c24ef003b
:103e40008c04a8008c84a80020002000004088007a
:103e500000248000700060000000e00007003200d5
:103e600010248000700060000000e00003003200b9
:103e700000012000002488009a04070040248000ec
:103e8000620060000000e000020032008ec0a90065
:103e9000a200370050248000610060000000e000b4
:103ea0000900320060248000610060000000e00032
:103eb0000500320046ff0700400020000040880057
:103ec0001000200050248800502480007000600002
:103ed0000000e000050032006024800070006000f7
:103ee0000000e0000100320071040700012480009e
:103ef00000042000008060000000e00003003200a9
:103f00000004200000248800d1060700502480000f
:103f1000640060000000e0001400320060248000b3
:103f2000640060000000e000040032001200200085
:103f30008000eb0030072000e80c07004000200064
:103f40005024880011c8bf000004e00003003200c4
:103f500011c8bf000040e90011e8b70011c8bf0058
:103f60000004e00001003a008101070051248000b4
:103f700000082000008060000000e0000600320021
:103f80006124800000082000008060000000e00044
:103f9000010032002a040700502480006200600003
:103fa0000000e0000c00320060248000620060002d
:103fb0000000e00008003200120020008000eb004a
:103fc000f0ff2700c50c07000080eb00702488007c
:103fd000200020005024880000408000e30f5000a3
:103fe00002003e008ec0a9004c0037006024800013
:103ff000680060000000e000470032000040eb0075
:10400000004f78003f0037005024800068006000b7
:104010000000e0003f003200902480000040780063
:104020000ee8b7000ec8bf000080fb004400de00b1
:10403000004078000fe8b70080002000502488007e
:104040000ec8bf00684060000004e00012003a00a3
:104050000fc8bf000081fb000fc8bf008080fb00bd
:10406000a09c2000008040009040780061c060006b
:104070000004a200e1406000a09c2000000041007c
:10408000e1c06000104178000204a100814071008d
:1040900001487800110037000fc8bf000081fb0005
:1040a0000fc8bf008080fb00609c200000804000a3
:1040b0009040780061c060000004a200e140600010
:1040c000609c200000004100e1c0600010417800c9
:1040d0000204a10081407100014878000fc8bf00b0
:1040e0000004e00002003a000a0407000400370060
:1040f0000001eb00e180200020072000770c070082
:104100001e4fe8001e407800e34f5000beff36000f
:1041100001003700000000008ec0a9000080fa00f6
:10412000000006000400fa0020479800314798007c
:104130003e4090000080fb00680060000000e0004e
:10414000030032008040eb002e4090007701070012
:104150003e4090000080fb00640060000000e00032
:104160000300320011c0b3002e4090006f01070021
:10417000a14a20002e4090000080fb00000040007b
:10418000008f40001e007800be409000014878007b
:104190000080fa00000006000800fa00204798009e
:1041a0003147980022079800634798003e409000ee
:1041b0000004e000070032002e4090000080fb0069
:1041c00080004000209b200000804000100f7800fd
:1041d000060037002e4090000080fb008000400069
:1041e000c09a200000804000100f78001e00780068
:1041f0000000e00002003a000000eb00370037004a
:10420000ae0090001e007800110098001e0078009b
:10421000ee409000014878001e00780010409000a9
:1042200002c4b300824060001e0078001140980074
:104230001e00780010409000804078000134a000fb
:104240001e007800114098001e0078001040900079
:10425000804078000174a0001e0078001140980092
:104260003e4090000004e0000e0032002e4090001e
:104270000080fb00ae4090008180fb000181400087
:10428000219b200081004100910078000120a200c4
:1042900000014000209b2000000041000108780040
:1042a0000d0037002e4090000080fb00ae409000d3
:1042b0008180fb0001814000c19a20008100410003
:1042c000910078000120a20000014000c09a200067
:1042d00000004100010878001e0078000080fa000c
:1042e000000006000400fa002047980031479800bb
:1042f0002e4090000004e00017003a00304080009b
:1043000081c0b3000148780030408000d19c20007b
:104310001100980030408000c1c0b30011409800e7
:104320003040800031408000914090000174a00036
:1043300011409800904d800041c0b300114098009a
:10434000904d8000914d8000914090000174a0003c
:10435000114098002e0037002e4090000080fb0096
:1043600000004000800078003e4090000080fb008c
:10437000008040004300dd008000780000a02000a5
:10438000008f40001e0078001040900080407800b0
:104390000124a0001e007800114098001e00780043
:1043a00010409000804078000174a0001e0078004a
:1043b000114098002e4090000080fb00000040005b
:1043c000800078003e4090000080fb0000804000ac
:1043d0004300dd00e400400000a02000008f40000a
:1043e0001e00780010409000804078000124a0005a
:1043f0001e007800114098001e00780010409000c8
:10440000804078000174a0001e00780011409800e0
:104410000080fa00000006000200fa00004f780059
:10442000a124800000022000008060000000e00065
:104430004d0032001e80fb0080004000209b2000c9
:1044400000804000100378001e80fb0080004000c8
:10445000209b200000804000100078001002be0069
:104460000004200001002000840378000502780089
:10447000800278008100780005806300810062007e
:1044800081017800000178000200be00008bbe00b0
:104490001e80fb0080004000209b20000080400028
:1044a000100278001e80fb0080004000209b20004e
:1044b00000804000100078001001be0000042000c1
:1044c000010020000000690081806900008abe00b0
:1044d0001e80fb009e80fb0001814000219b20008c
:1044e00081004100910078000120a20000014000fd
:1044f000209b200000004100010878001e80fb0086
:1045000080004000209b2000008040009000780048
:104510001e80fb0000014000209b200000004100a5
:1045200010007800104090000044b20090409800c5
:104530001e80fb0080004000209b20000080400087
:10454000900078001e80fb0000014000209b2000ae
:1045500000004100100078001041900000c4b3003a
:1045600000406900904098000080fa0000000600ba
:104570000000fa0013c8bf000004a2000004e0001d
:104580003400320010c0b30013e8b70014c8bf00f5
:104590000004a2000004e0002e00320010c0b300ae
:1045a00014e8b70009c8bf00e24f50000c003a0001
:1045b000904d80008040eb0001487800904d8000d5
:1045c00081c4b30011409800904d8000914d80004f
:1045d000914090000174a000114098001d00370028
:1045e00009c8bf00e14f50001a003a001068ef0000
:1045f0002040800081c0b300014878002040800046
:10460000d19c2000110098002040800041c0b300e0
:10461000114098002040800021408000914090008f
:104620000174a0001140980010c0b30010e8b7005a
:104630003040800081c0b3000148780030408000e5
:10464000d19c2000110098003040800001c8b300c8
:10465000114098000080fa00000006000000fa00f7
:104660001568ef001668ef0009c8bf00e24f500060
:104670000f003a003040800081c0b300014878004c
:1046800030408000619d2000110098003040800083
:1046900081c4b30011409800304080003140800058
:1046a000914090000174a000114098001d00370057
:1046b000309d20001080fb00419d20009180fb0078
:1046c000c808dd000100700080007800e04d800027
:1046d000808f500007003100309d20001080fb00cb
:1046e000419d20009180fb00c808dd0001007000a2
:1046f000e04d880096000700904d8000619d2000ed
:1047000011009800904d800081c4b30011409800c2
:10471000904d8000914d8000914090000174a00068
:10472000114098000080fa00000006000400fa0022
:10473000204798003147980000a02000000f780023
:104740002e4090000080fb000000400080007800b8
:104750003e4090000080fb00008040004300dd00f0
:104760001e0f40001e0078009000780001f0a100ac
:10477000010878003e4090000004e00007003a0085
:104780002e4090000080fb0080004000c09a200076
:10479000008040001e087800060037002e40900080
:1047a0000080fb0080004000209b20000080400033
:1047b0001e0878001e0078009000780001e0a1003b
:1047c000010878009e007800648040009000780026
:1047d00001e0a000010878000080fa000000060057
:1047e0000000fa0094a4a900d14d80000008200028
:1047f000008060000000e00027003a00009c2000dc
:104800009040780000c8b30000c060000004e000e1
:104810000a00320020c0b30009e8b70016c8bf0084
:104820000004a2000004e000010032008bff07003a
:104830001468ef001368ef00430037003040800039
:1048400081c0b3000148780030408000d19c200036
:104850001100980030408000c1c0b30011409800a2
:104860003040800031408000914090000174a000f1
:1048700011409800904d800041c0b3001140980055
:10488000904d8000914d8000914090000174a000f7
:10489000114098002c003700d09c200090407800f8
:1048a00000c8b30000c060000004e0000f00320048
:1048b00010c0b30009e8b70015c8bf000004a2008b
:1048c0000004e0000100320064ff07001468ef00fc
:1048d0001368ef0012c8bf000004a2000004e0004b
:1048e0001900320022ff07001700370020c0b30074
:1048f00009e8b7003040800081c0b300014878006b
:1049000030408000d19c2000110098003040800091
:1049100041c0b30011409800304080003140800019
:10492000914090000174a000114098001468ef00bd
:104930001368ef0012c8bf000004a2000004e000ea
:10494000010032000aff07000080fa0000000600a4
:104950000200fa0080c0b300004f7800e04d8000f4
:10496000e70f50000d003e00e04d8000004f780042
:1049700008c8bf000004e00003003a0010c0b30004
:1049800008e8b7000500370008c8bf00e14f500035
:1049900002003a0020c0b30008e8b700e14d8000f3
:1049a0001e80fb0000805000e04d8800904d80008c
:1049b0001e487800609d200050408800d04d800047
:1049c000610060000000e00017003a0009003700b5
:1049d00051408000c04d800010417800824878002e
:1049e0008100e800514088000000e800c04d8800c8
:1049f0001e4fe9001e4078000004e000f4ff3a007a
:104a00000c00370051408000c04d800010417800fc
:104a1000824878008100e800514088000000e800ea
:104a2000c04d88001e4fe9001e4078000004e000e1
:104a3000f4ff3a000080fa00000006000200fa00cd
:104a400020408000104f78009e80fb00004e8000c8
:104a50004800de00134e8000f20f2000028161004a
:104a60004811dd0002007000808f50000800360001
:104a7000004e80004800de00124e8000f10f200042
:104a800081006100c808dd0001007000004f78005f
:104a9000004e80004800de00124e8000f10f200022
:104aa00081006100c808dd0001007000800078000e
:104ab0001e80fb0000805000f10f2000810060008c
:104ac000c808dd00034e8000f20f20000281610063
:104ad00082807000014e8800c800de00f00f2000c8
:104ae00000806000124e800001f02f008100610004
:104af00001007000104e88000040eb001047980045
:104b00000c003700f04d80009e4090000181fb00ba
:104b1000619d2000810041009140780001487800ab
:104b20000000e800f04d88001e4090000040e800c2
:104b3000104798001e4090009e4f5000f1ff390032
:104b4000004e80004800de00124e8000f10f200071
:104b500081006100c808dd00010070000000e00075
:104b60001e0032003040800081c0b3000148780050
:104b700030408000619d200011009800204080009e
:104b80009000780000002400008060000000e00039
:104b900009003a003040800081c4b3001140980001
:104ba0003040800031408000914090000174a000ae
:104bb00011409800300037003040800081c0b300c1
:104bc00011409800304080003140800091409000ba
:104bd0000174a00011409800270037003040800089
:104be00081c0b3000148780030408000d19c200093
:104bf000110098003040800041c0b300114098007f
:104c00003040800031408000914090000174a0004d
:104c100011409800104e80004800de00224e8000b7
:104c2000f10f200081006100c808dd000100700064
:104c30000000e00008003200104e80004800de0056
:104c4000224e8000f10f200081006100c808dd00c5
:104c50000100700000000100004e80000070a10003
:104c6000004e880012c8bf000004a2000004e0004b
:104c7000010032003efe07000080fa00000006003e
:104c80000200fa00d04d80000070a000d04d8800d6
:104c9000420020008000eb00c04a2000d8fa070044
:104ca000020320008000eb0000a02000d4fa0700df
:104cb0009424a8000040eb00004f78000b00370060
:104cc0009e80fb00609c2000008040008040eb0044
:104cd000014878009e80fb00a09c200000804000de
:104ce0008040eb00014878001e4fe8001e4078002d
:104cf000e24f5000f2ff3600220020008000eb005f
:104d0000a09a2000befa07009424a90080a02000e9
:104d1000904d880000a020002040880020408000a6
:104d200030408800f09c20001040780002e8b70076
:104d300002c8bf000004e00003003a0000012000a8
:104d4000004088000600370012002000218020006b
:104d500010002000610907000002200000408800c8
:104d60000080fa00000006000000fa00d09c20003d
:104d70009040780000c8b30080cf500047003a0050
:104d8000a09b200001ccb30001487800009d2000ca
:104d9000104078000080fb00e20f50000900320054
:104da000e30f500023003200e10f500037003a00bb
:104db00040cd2900c04d880020012000e04d880032
:104dc00036003700f09c2000104078000004e0001e
:104dd00014003a00f09c2000104078000080fb0096
:104de0000000400080007800e0d5290000804000ed
:104df00010007800c04d8800c04d80000080e800a1
:104e000090407800c09b200001487800c04d800091
:104e10006300400090407800d09b2000014878005b
:104e20001e003700a09b20008040eb000148780066
:104e30001a003700f09c200010407800e24f50002c
:104e40000e003e00f09c2000104078000080fb0027
:104e5000000040008000780000d62900008040005b
:104e600010007800c04d8800c04d800010407800d0
:104e70000080fb00e04d880008003700a09b200068
:104e80008040eb000148780004003700a09b200020
:104e90008040eb0001487800000000000080fa002c
:104ea000000006000200fa00609d20008040eb0038
:104eb00001487800709d20008040eb000148780098
:104ec000d09c2000904078007fc060000080fb00f4
:104ed000e10f500011003200e20f500013003200c9
:104ee0000000e00047003a00d04d80000070a000b4
:104ef000d04d88000cc8bf000004e0003a0032002a
:104f0000609d200010407800804078000114a000cf
:104f1000609d2000014878003a003700d04d8000a5
:104f20000070a000d04d880036003700d04d8000c2
:104f30000070a000d04d8800109d20001040780027
:104f40006f4060000004e00029003200109d200046
:104f50009040780000c8b30000c060000004e0008a
:104f600009003a00109d2000904078006fc060005a
:104f70000080fb0080004000c09a200000804000bc
:104f8000100f780008003700109d20009040780036
:104f90006fc060000080fb0080004000209b20006c
:104fa00000804000100f78001e007800900078000c
:104fb00000002800008060000000e0000e003200c9
:104fc0001e00780090007800004020000080600003
:104fd0000000e0000a003200609d200011c0b30014
:104fe0000148780007003700000000000500370086
:104ff000000000000300370000000000010037003f
:1050000000000000d14d80000008200000806000fa
:105010000000e00008003200609d2000c04d8800c4
:10502000d04d80000000a000d04d8800c09b200023
:1050300021c0b300014878000080fa00000006009b
:105040000000fa0050258000620060000000e000cf
:1050500013003200204080009040900000c8b30050
:1050600080cf50000d003a00904d8000904090009d
:1050700040c8b30080cf500008003a0020408000b4
:10508000c1c0b30011409800204080002140800042
:10509000914090000174a00011409800aa24a9003a
:1050a00000082000502488000080fa00000006005c
:1050b0000000fa008284a80000012000502488002b
:1050c00010c0b3000de8b7001c68ef000001eb0052
:1050d0008000eb0050072000800807000080fa00e5
:1050e000000006000000fa000d68ef000001eb0070
:1050f0008000eb0040072000780807008284a900a8
:1051000000012000002488001c68ef000080fa00e5
:10511000000006000000fa00d0c2b30011e8b7009a
:105120000ec8bf000080fb000020a1000000e000ce
:105130001f003a000ec8bf000080fb004200de00e6
:10514000004078000080fb00c200dd0000a02000cd
:1051500000804000204088002040800030408800cf
:10516000304080000020a2003040880020408000b5
:105170009000780000c02300808060000040230081
:10518000808f500008003a002040800010009000fe
:105190008200200080007800d09c200091f9070058
:1051a0000b000700080037003d000700060037002d
:1051b0000ec8bf000080fb000020a100e80f5000d7
:1051c00001003a00530007000080fa0000000600ca
:1051d0000000fa000868ef001268ef001568ef00a1
:1051e0001668ef001068ef000968ef00904d80002e
:1051f000914d8000914090000174a10011409800f1
:10520000904d80000020a200904d8800904d8000bd
:10521000914d8000914090000174a10011409800d0
:10522000904d80000020a200904d8800304080000a
:1052300031408000914090000174a100114098001d
:10524000a09b20008040eb00014878000000eb00ac
:10525000e04d8800009c20008040eb000148780071
:10526000014e8000f00f200000806000004e88009a
:10527000114e800000f02f0000806000104e88006a
:10528000830007000001eb008000eb0030002000ed
:105290001208070052fd07000080fa000000060017
:1052a0000000fa0009c8bf00e24f500002003a00b7
:1052b000e2fd0700150037000968ef0010c8bf00c5
:1052c0000004a2000004e0000f0032003040800023
:1052d00081c0b3000148780030408000d19c20009c
:1052e0001100980030408000c1c0b3001140980008
:1052f0003040800031408000914090000174a00057
:1053000011409800010037001068ef000080fa009b
:10531000000006000200fa00904d800010007800a6
:105320004e00de0061406000004f7800904d80002c
:105330000020a200904d880000408000e80f50003f
:105340000e003a00f09c2000104078008080fb00a6
:10535000f007200000806000b0248800b0248000a6
:105360000000e0000300320000012000004088003f
:1053700002003700400020000040880009c8bf003c
:10538000e14f500025003a00904d8000619d2000c3
:10539000110098006efd070008c8bf00e24f5000e2
:1053a00009003a00904d800041c0b30011409800c0
:1053b000904d8000914d8000914090000174a000bc
:1053c00011409800300037001e4078000004e000d3
:1053d00009003a00904d800081c4b300114098004c
:1053e000904d8000914d8000914090000174a0008c
:1053f0001140980024003700904d800081c0b30018
:1054000011409800904d8000914d80009140900097
:105410000174a000114098001b003700009c200080
:105420009040780000c8b30000c060000004e000b5
:1054300014003200104e80004800de00224e800032
:10544000f10f200081006100c808dd00010070003c
:105450000000e00008003200104e80004800de002e
:10546000224e8000f10f200081006100c808dd009d
:105470000100700000000100004e80000070a100db
:10548000004e88000968ef000080fa000000060066
:105490000000fa00d09c2000104078000046b200c6
:1054a0000004e00051003a00e09c20001040780029
:1054b0000080fb00cf80de00b2002000030020004f
:1054c000820f5000838f58004a003e0000600100a8
:1054d0002100370022003700480037002000370045
:1054e00046003700060037000b0037003a0037004f
:1054f0000d0037000a0037001b0037002a00370074
:10550000d04d80000070a000d04d880080002000a9
:10551000004088003a00370013fe070038003700cb
:10552000d7fd07003600370020802000c04d8800de
:10553000d04d80000000a000d04d8800c09b20000e
:1055400011c0b30001487800d04d80000070a00069
:10555000d04d88002a00370052fe0700280037008f
:105560002900070026003700109d20001040780019
:105570008080fb00a09a200000804000c04d880081
:10558000d04d80000000a000d04d8800c09b2000be
:1055900011c0b30001487800d04d80000070a00019
:1055a000d04d880016003700d04d80000070a0005c
:1055b000d04d8800109d2000104078000081fb0035
:1055c000f09c200090407800a09a2000000041004c
:1055d000014878000a0037000001eb008000eb0072
:1055e000200020003d0707000500370000000000f4
:1055f0000300370000000000010037000000000039
:105600000080fa00000006000600fa00f09c20006e
:1056100010407800e14f500010003a00d09c20006c
:10562000104078007f4060000004e0000b003a006a
:10563000d04d80000070a000d04d8800e09c20007c
:1056400010407800e34f500003003a0010c0b30050
:105650000ce8b700010037000c68ef00f09c200058
:10566000104078000004e000f7003a00d09c2000d1
:10567000104078007f406000e24f5000f2003a0096
:10568000109d2000104078006f4060000004e00092
:10569000ed003200109d2000904078006fc0600047
:1056a0000080fb00e20f5000e7003c00014080005a
:1056b00000022000808f5000e3003a00d04d8000af
:1056c0000070a000d04d8800109d20009040780010
:1056d00000c8b30000c060000004e00011003a0000
:1056e000109d2000104178006f4061000080fb0099
:1056f00080004000c09a200000804000100f780019
:10570000109d2000904078006fc060008080fb00fa
:10571000a09c200000804000104078004047980086
:1057200010003700109d2000104178006f4061008c
:105730000080fb0080004000209b20000080400093
:10574000100f7800109d2000904078006fc060001e
:105750008080fb00609c20000080400010407800aa
:10576000404798004e409000614060000004e00017
:1057700004003a001e0078000020a100000f78000d
:10578000030037001e0078000020a000000f780002
:10579000109d20009040780000c8b30000c0600059
:1057a0000004e0000a003a00109d2000104178003b
:1057b0006f4061000080fb009e0078000001400007
:1057c000c09a20000000410001087800090037005d
:1057d000109d2000904078006fc060000080fb00aa
:1057e0009e00780000014000209b20000000410046
:1057f00001087800e09c200010407800e34f500042
:105800002c003a001e00780090007800000028006c
:10581000008060000000e00019003200109d2000b0
:105820009040780000c8b30000c060000004e000b1
:105830000a003a00109d2000104178006f4061007e
:105840008080fb00a09c20000080400090407800f9
:105850000114a0000148780009003700109d2000c5
:10586000904078006fc060008080fb00609c20004a
:1058700000804000904078000114a00001487800aa
:105880001e00780010409000804078000124a000a5
:105890001e007800114098001e0078001040900013
:1058a000804078000174a0001e007800114098002c
:1058b000650037001e0078000020a200000f78006d
:1058c0001e00780090007800000028000080600032
:1058d0000000e000110032001e007800104090002f
:1058e000804078000174a1001e00780011409800eb
:1058f0001e00780010409000804078000164a000f5
:105900001e00780011409800220020009e007800c0
:105910005000200071060700060037001e007800c6
:1059200010409000804078000164a0001e007800c4
:10593000114098001e0078000020a200000f78009f
:105940004e409000624060000004e00006003a0013
:105950001e007800900078000000280000806000a1
:105960000000e00024003200109d200090407800ec
:1059700000c8b30000c060000004e0000a003a0064
:10598000109d2000104178006f4061008080fb0076
:10599000a09c200000804000904078000114a100ed
:1059a0000148780009003700109d200090407800e1
:1059b0006fc060008080fb00609c20000080400081
:1059c000904078000114a100014878001e00780082
:1059d00010409000b2c3b300824060001e00780007
:1059e00011409800220020009e0078005000200006
:1059f0003a060700060037001e00780010409000ad
:105a0000b2c3b300824060001e00780011409800cd
:105a1000a14a2000109d2000104178006f406100d5
:105a20000080fb000000400000804000100798004c
:105a30001e00900010407800804078000114a10002
:105a40001e009000014878000080fa000000060067
:105a50000000fa00c0408000d1408000610040009a
:105a6000e0804800c0408800d14088000dc8bf00d9
:105a70000004a2000004e000080032001cc8bf00bf
:105a80000040e8001ce8b7001cc8bf000004e000ac
:105a900002003a0000c0eb001ce8b7000080fa00ea
:105aa000000006000000fa00c0408000d1408000e5
:105ab0000080fa00000006000000fa00d09c2000e0
:105ac000104078007f406000e14f500078003a00bd
:105ad000d09c20001040780002c6b30082406000d5
:105ae00000c2b30080cf500073003a00109d200028
:105af000104078000004e00004003200109d2000f7
:105b000010407800e14f50006d003a00e09c20000a
:105b1000104078000080fb0001022000810f50003f
:105b20002000320001022000810f500005003c00df
:105b30000000e0000a003200e10f500013003200c4
:105b40006000370011022000810f50004300320036
:105b500021022000810f5000480032005900370018
:105b6000209a2000c04d880080002000e04d880071
:105b7000d04d80000000a000d04d8800d04d8000a6
:105b80000070a000d04d88004e003700209a200001
:105b9000c04d8800d04d80000070a000d04d88001e
:105ba00048003700309d20001080fb00419d200000
:105bb0009180fb00c808dd0001007000f10f20009b
:105bc00001016000119c200091417800e0c161005a
:105bd00002c1710082487800c800de00209c2000cd
:105be00010417800604161008140710001487800f7
:105bf00000992000f10f200001016000e19b2000ce
:105c000091417800e0c1610002c1710082487800d2
:105c1000c800de00f09b2000104178006041610068
:105c20008140710001487800309c2000904078004d
:105c3000e0c0600001487800409c2000904078005f
:105c4000e0c0600001487800009c2000904078008f
:105c50000174a000014878001a0037000099200064
:105c6000c04d880070002000e04d8800a09b2000ff
:105c700011ccb3000148780012003700f09c2000de
:105c80001080fb00019d20009180fb00c808dd0012
:105c900001007000004078002ae8b700d04d800075
:105ca0000070a000d04d8800000000000500370003
:105cb0000000000003003700000000000100370072
:105cc000000000000080fa00000006000000fa005a
:105cd00000b0240001002000804c8800914c880016
:105ce000409920008040eb00014878005099200046
:105cf0008040eb00014878006099200081c0b3002b
:105d0000014878001e68ef0051c1b30010c0b30015
:105d100004f90700d1c1b30020c0b30001f90700a6
:105d200003c4b300029520008040eb0020c0b30004
:105d300019f90700304188002828ef001f68ef009c
:105d40000080fa00000006000600fa00000f78004c
:105d500011079800220798001e007800e50f5000f8
:105d600012003a00304180009e009000808f500069
:105d700006003a0003c4b300029520008040eb0007
:105d800020c0b30004f90700304188004041800082
:105d90009e009000808f500002003a001f68ef00c4
:105da0002468ef0010c0b300010037000040eb0092
:105db0000080fa00000006000400fa00000f7800de
:105dc000214798001e68ef00304180000000e0008d
:105dd000060032003041800090007800000028006a
:105de000008060000000e00022003a0030418000a6
:105df000904078002e40900080cf5000030031008a
:105e00003041800090407800214798001e68ef00e4
:105e10000d0037001ec8bf000080fb001e004000c0
:105e2000e1812000914078000181fb000195200074
:105e30008100410091407800014878001ec8bf00f1
:105e40000040e8001ee8b700e181200091407800a2
:105e50002e40900080cf5000eeff390003c4b30005
:105e6000029520008040eb0020c0b300caf8070074
:105e7000304188001ec8bf000080fa000000060004
:105e80000400fa00000f7800214798001fc8bf00e7
:105e90000004e00009003a009e00780001418800fb
:105ea000ae409000428220000149780010c0b3004b
:105eb00025e8b70010c0b3001fe8b7000080fa0063
:105ec000000006000600fa00200798001fc8bf0067
:105ed0000004e0001f003a000040eb00004f780093
:105ee000ae009000110798001e4fe8001e40780099
:105ef000e14f40000c0032001e009000104078007e
:105f00000080fb000000ea004f00de000040780047
:105f10009e0090008100e800110798000004e00056
:105f2000f1ff3a0001003700000000002e00900051
:105f3000004188009e40780042822000014978009c
:105f400010c0b30025e8b70010c0b3001fe8b700c9
:105f500001003700000000000080fa000000060089
:105f60000600fa00200798001fc8bf000004e000e8
:105f70001e003a000040eb00004f7800ae00900099
:105f8000110798001e4fe8001e407800e14f4000c6
:105f90000c0032001e009000104078000080fb00d2
:105fa0000000ea004f00de00004078009e009000f4
:105fb0008100e800110798000004e000f1ff3a00ba
:105fc00001003700000000002e0090000041880012
:105fd0009e40780042822000014978002568ef0049
:105fe00010c0b3001fe8b700010037000000000038
:105ff0000080fa00000006000200fa004041800024
:106000000000e0000600320040418000900078006f
:1060100000002800008060000000e00060003a00fe
:106020001fc8bf00e34f500001003a001f68ef0097
:106030001fc8bf000004e0005b0032001fc8bf00a3
:10604000e24f500009003a008041eb000001eb00f4
:1060500011c0b30020c0b3004ff8070040418800d2
:1060600030c0b3001fe8b700500037001fc8bf00a2
:10607000e14f50004d003a004182200091407800ed
:1060800000c4b30080cf50000300360000c4b3004a
:10609000004f7800030037004182200091407800d3
:1060a000014f780024c8bf001e40500024e8b7000c
:1060b00000912000104188009e4078001147980010
:1060c00025c8bf000004e0001f003a000d003700a3
:1060d0001041800001418000914078000148780023
:1060e000104180000000e80010418800004180005d
:1060f0000000e800004188001e4090000040e900d8
:10610000104798001e4090000004e000f0ff3a00a5
:10611000100037001041800001418000914078005c
:1061200001487800104180000000e800104188001c
:10613000004180000000e800004188001e409000ff
:106140000040e900104798001e4090000004e00065
:10615000f0ff3a0024c8bf000004e00009003a0044
:1061600000c4b3009e40780080cf500003003a0086
:1061700020c0b3001fe8b7000200370030c0b300f2
:106180001fe8b7009e4178000291200011c0b300c3
:1061900020c0b30000f8070040418800030037002a
:1061a0000000000001003700000000000080fa003d
:1061b000000006000200fa000000eb00000f78006b
:1061c00010002000000f78001e00780000407800ca
:1061d0000080fa00000006000200fa000000000043
:1061e0003104800000002400008060000000e00016
:1061f000fbff3200b0118000004f780087c0a9007b
:106200001e4078000080fa00000006000000fa003e
:1062100020022000c01188003022ef003062a80068
:106220003222ef0031e2a8003342a80087c0a90063
:106230000080fa00000006000000fa00310480002f
:1062400000002400008060000000e0000200320036
:1062500010c0b300010037000040eb000080fa00de
:10626000000006000400fa00100798000200370042
:106270001e4078000e0007001e00900010407800bd
:10628000004f78001e80fb000000ea004f00de0097
:10629000004078009e0090008100e80011079800ff
:1062a0000004e000f2ff3a000080fa00000006005f
:1062b0000200fa00004f78001e00fb00a0118800c9
:1062c000000000009111800000102000008060009c
:1062d0000000e000fbff32000080fa000000060032
:1062e0000400fa00204798000040eb00004f7800bf
:1062f000ae409000114798009e40900030c6b30019
:1063000080cf50000b0036001e4090000080fb0044
:10631000c200de00b04721000008b8000100d10033
:10632000004078000043b000e1ff070010c0b30058
:10633000004f78001e4090000080fb00c200de008d
:10634000b04721000008b8000100d100804078006b
:10635000c00920000088b9000000780000407800e3
:106360009e40900000c04000104798001e409000e2
:10637000e94f500003003e001e407800e14f5000fe
:1063800008003a001e4090008080fb00d0cc2c001a
:106390000008b8004308de00004078000043b00069
:1063a000c3ff07001e4090008080fb00d0cc2c0073
:1063b0000008b8004308de0080407800600f20002d
:1063c0000088b90000007800004078009e409000ee
:1063d00000c04000104798001e4090000043b000ed
:1063e000b3ff07000080fa00000006000400fa0076
:1063f000100798009e009000010f78001e0090008a
:106400004480de006f006000100798009e0090003e
:1064100080dd29000080400010407800a4ff0700c4
:106420009e0078006f806000100798009e0090002a
:1064300080dd290000804000104078009cff0700ac
:106440000080fa00000006000400fa00100798001f
:106450001e0090004c00de00000f780080dd290057
:106460001e0040001040780091ff07001e009000c1
:106470004800de006f0f600080dd29001e00400034
:10648000104078008aff07001e0090004400de00e4
:106490006f0f600080dd29001e0040001040780072
:1064a00083ff07001e0090006f0f600080dd290051
:1064b0001e004000104078007dff07000080fa00b9
:1064c000000006001800fa00889fbe008a9fbe00e8
:1064d0008c9fbe0020079800310798002e00900086
:1064e000be0090004c08de0001002000008fbe00be
:1064f00080dd29001e004000104078006cff07007e
:106500002e009000be0090004808de0000007800d9
:106510006f0060008000eb00510798004007980072
:106520004e019000de019000028fbe0080dd290048
:106530001e004000104078005dff07002e00900014
:10654000be0090004408de00000078006f0060008c
:106550008001eb0073079800600798006e019000bf
:10656000fe019000028fbe0080dd29001e00400069
:10657000104078004eff07002e009000be009000f3
:106580004008de00000078006f0060008001eb0032
:10659000130f9800000f98000e0990009e099000bc
:1065a000028fbe0080dd29001e00400010407800f0
:1065b0003fff07002e009000be009000c409dd00e0
:1065c0004c00de0000807100cc08de000000780086
:1065d0006f0060008000eb00310f9800200f9800e2
:1065e0002e099000be099000028fbe0080dd2900b8
:1065f0001e004000104078002dff07002e00900084
:10660000be009000c809dd004800de000080710077
:10661000c808de00000078006f0060008006eb0014
:10662000000678000c8fbe0080dd29001e004000af
:10663000104078001eff07002e009000be00900062
:106640004c09dd004400de0000007100c408de00db
:10665000000078006f0060008005eb000005780006
:106660000a8fbe0080dd29001e0040001040780027
:106670000fff07002e009000be0090000000780081
:106680006f0060008004eb0000047800088fbe00fb
:1066900080dd29001e0040001040780004ff070044
:1066a0004f06be004f05be004f04be000080fa003a
:1066b000000006000200fa00004f780060c6b30038
:1066c0009e40780080cf5000020034000040eb0074
:1066d0002500370000c6b3009e40780080cf5000f0
:1066e000040034009e40780090cab30000c040000f
:1066f0001d00370060c4b3009e40780080cf50007a
:10670000020034000040eb001700370000c4b30063
:106710009e40780080cf5000040034009e407800f6
:1067200090ccb30000c040000f00370090c3b3000e
:106730009e40780080cf5000020034000040eb0003
:1067400009003700f0c2b3009e40780080cf5000af
:10675000040034009e40780000cdb30000c040002b
:10676000010037000040eb000080fa000000060046
:106770000400fa00204798002e4090006f4f600000
:106780001e407800e94f5000030034001e4078009e
:106790007043b000020037001e4078000043b00094
:1067a0000080fa00000006000000fa00901180004e
:1067b000620060000000e000010032003222a90007
:1067c0000080fa00000006000000fa00a2000700a6
:1067d0000040fe0051248000000220000080600084
:1067e0000000e00002003a0010c0b30041000700c2
:1067f000d200070010c0b3000080fa0000000600bd
:106800000000fa000cc8bf000004e00036003200af
:106810000dc8bf000004e0003300320040248000b7
:10682000620060000000e000010032008824a9003e
:10683000750007000004200000248800000000000c
:106840000124800000042000008060000000e000bf
:10685000fbff32000004200000248800000000003c
:106860000124800000042000008060000000e0009f
:10687000fbff32000004200000248800000000001c
:106880000124800000042000008060000000e0007f
:10689000fbff32009444a80000042000002488007c
:1068a000000000000124800000042000008060003f
:1068b0000000e000fbff32000004200000248800fc
:1068c000000000000124800000042000008060001f
:1068d0000000e000fbff32009444a90057000700cd
:1068e00010c0b300010037000040eb000080fa0048
:1068f000000006000400fa002047980040248000b1
:10690000610060000000e0000b00320040248000c5
:10691000620060000000e00007003a001cc8bf00f1
:10692000e34f500004003600202480004300de00c6
:1069300061406000320037002e4090000004e0000b
:106940001d0032008824a9008804a8002e0007003a
:106950000040eb00004f78000900370000042000e1
:1069600000248800000000000124800000042000b2
:10697000008060000000e000fbff32001e4fe800d6
:106980001e407800e44f5000f4ff36000040eb005a
:106990001047980020248000680060000000e0009c
:1069a0000200320010c0b300104798002300070017
:1069b0001e409000120037004024800061006000fb
:1069c0000000e00002003a0000c0eb000c003700bd
:1069d00040248000620060000000e00002003a00f5
:1069e000e0cfb300060037001cc8bf00e34f5000e3
:1069f00002003e00d0cfb30001003700c0cfb3008b
:106a00000080fa00000006000000fa003868ef007d
:106a10001000fc00f10480000004200000806000f1
:106a20000000e0000200320010c0b30038e8b700f8
:106a30009ec0a9000080fa00000006000000fa00d5
:106a400038c8bf000004e000010032009ec0a8006a
:106a50000080fa00000006000400fa001e00fc009e
:106a600011028000000e200000806000804188003c
:106a700011028000000e200001007000100288004a
:106a800040092000100798000000eb00000f78007c
:106a90000e0037001e009000900078001e00780065
:106aa00000014000e09d2000000041000108780046
:106ab0001e0090008000eb00010878001e0090008e
:106ac0000080e800100798001e0fe8001e00780004
:106ad000e50f5000efff36006024800090418800f1
:106ae0008c24ef0010248000a04188008224ef0055
:106af000700680004800de00674060000080fb00f8
:106b0000b04188000001200000248800000220001d
:106b1000502488008ec0a9008284a80071068000dd
:106b2000f08f2f000080600000a0a0007006880099
:106b30009ec0a8000080fa00000006000400fa00d1
:106b400040092000100798000000eb00000f7800bb
:106b50000b0037001e00780080004000e09d200000
:106b600000804000900078001e009000010878002e
:106b70001e0090000080e800100798001e0fe8003b
:106b80001e007800e50f5000f2ff360090418000b3
:106b900060248800a041800010248800b04180005b
:106ba00000407800674060000080fb0067006000e4
:106bb0004800dd0072068000f18f2f008100610027
:106bc000010070007006880011028000f0f12f00b3
:106bd000808060008041800001007000804188005a
:106be00080418000100288000080fa00000006004a
:106bf0000200fa0090118000680060000000e000d0
:106c000002003200b0118000004f78009011800027
:106c1000640060000000e00002003200b01180005b
:106c2000004f780090118000620060000000e000da
:106c3000010032003222a9000080fa0000000600a4
:106c40000000fa00213a8000f0f32f00008060007d
:106c5000203a88000100370000000000113a80004f
:106c600000022000008060000000e000faff320017
:106c700040a7a900b1368000f00f2c008080600092
:106c80000050200001007000b036880031358000cf
:106c900000fc2f00008060008001b30030358800c8
:106ca000f0c2a900f0e2a900f102a900f122a900b6
:106cb000d9e2a900e882a900e8a2a900d022a80090
:106cc000d062a800e102a800e122a800020420008e
:106cd0008000eb0000842000c9f2070090168000bd
:106ce000680060000000e0000a003a00001a20007e
:106cf000c01188003022ef003062a8003222ef007d
:106d000031e2a8003342a80087c0a9003222a900be
:106d10000900370020022000c01188003022ef0057
:106d20003062a8003222ef0031e2a8003342a8000e
:106d300087c0a9003222a9000000eb00c4010700af
:106d4000a3f30700960007003e01070060da290060
:106d5000ec000700c1118000001a2000808f500055
:106d600003003a0070db2900e6000700040037004a
:106d700070dc2900e300070001003700000000007c
:106d80000df4070010000700901180000000d100f2
:106d9000614060000080fb004f00dd00e1168000d4
:106da00001f0a10001007000e016880011178000ba
:106db00000202000008060000000e000efff3a00ab
:106dc0008bff0700eeff37000000fa00881f7800f5
:106dd00000408000ff0f50006b0036004024800010
:106de000620060000000e00069003a003dc8bf009a
:106df0000004e0000a003a0001c4b300008820004b
:106e0000edfb07003be8b7003bc8bf000004e00013
:106e10000300320010c0b3003de8b7003c68ef004b
:106e20003dc8bf000004e000230032009111800043
:106e300000102000008060000000e0001e00320012
:106e40003cc8bf008080fb0000882000008040001c
:106e50001040780016fd0700a117800000042000f4
:106e60000080600000f0a7000000ea000000e900d8
:106e70004f00de00004078000080fb0061006000f1
:106e80004600dd00a11780000160a1000100700034
:106e9000a01788003cc8bf000040e8003ce8b700ed
:106ea000c1832000914078003bc8bf0080cf5000d4
:106eb00001003a003d68ef00dffc07000004e0003d
:106ec00015003200a183200091407800e0c3b30098
:106ed00080cf500010003e003ac8bf000084fb0085
:106ee000bdfc0700804078000084200000004400c2
:106ef000014878003ac8bf000040e8003ae8b7000f
:106f00003ac8bf008080fb00008420000080400061
:106f10008040eb00014878001fc8bf000004e0007b
:106f200017003a003ac8bf000004e0001400320025
:106f30003ac8bf008040780000842000d0fb0700e2
:106f4000a1178000002020000080600000f0a70052
:106f50000000ea000000e9004f00de000040780079
:106f60000080fb00610060004900dd00a117800087
:106f70000190a10001007000a01788003a68ef009e
:106f80001dfc07000300370000000000010037006f
:106f9000000000004f0478000080fa0000000600a6
:106fa0000000fa000117800000f02f000080600050
:106fb00000178800f002a900f022a900e822a90029
:106fc000f402a900f422a900ec22a9000050230039
:106fd000c1002000100107008040eb0080c3b30017
:106fe000110007008040eb0080c0b3000e000700d6
:106ff0008040eb0010c0b3000b0007008040eb00a6
:1070000060c0b300080007008040eb00c0c0b300c0
:107010000500070000b82b0001002000fe0007005b
:107020000080fa00000006000400fa0020479800e3
:107030003147980001178000f00f20000100700018
:1070400000178800f422a800f402a900211780008c
:1070500000f02f000080600020178800ec22a800bc
:107060000000000000000000000000001017800079
:107070004700de0061406000004f7800ec22a9006c
:107080001e4078000004e000f4ff3a000117800081
:1070900000f02f000080600000178800f422a90093
:1070a0003e4090000080fb000000ea004f00de0040
:1070b000004078000080fb0061006000a1178000a4
:1070c0000100a10001007000a017880021178000b6
:1070d00000f02f00808060002e4090000080fb00b8
:1070e0000100700020178800ec22a80000000000ba
:1070f0000000000000000000ec22a9000080fa005f
:10710000000006000400fa0010079800470037004e
:107110001e009000104f78001e00fb00eb0f400097
:107120002f003200eb0f40000c003c00f70f400036
:1071300019003200f70f400003003c00ff0f400031
:10714000120032002c003700f30f4000150032000f
:10715000ed0f40001600320027003700e60f400018
:1071600016003200e60f400003003c00ea0f40002a
:107170001e00320020003700e50f400015003200ed
:10718000e40f4000100032001b0037000040eb000d
:10719000004f78001800370010c0b300004f78008f
:1071a0001500370020c0b300004f780012003700f0
:1071b00030c0b300004f78000f00370040c0b3006c
:1071c000004f78000c00370050c0b300004f78002b
:1071d0000900370060c0b300004f78000600370098
:1071e00070c0b300004f780003003700f0ceb3004a
:1071f000004f7800000000001e407800ea4f500069
:1072000004003a008040eb0000ccb30086ff07008a
:10721000030037001e40780011c0b30082ff070052
:107220001e0090000000e800100798001e0090006b
:10723000104078000004e000b5ff3a000080fa003a
:10724000000006000200fa008040eb0000c4b3001a
:1072500075ff07000000eb00000f78000600370004
:1072600060d629001e0040001040780011c0b30015
:107270006dff07001e0fe800f00320009e0078005d
:10728000808f5000f6ff34008040eb0000c8b30050
:1072900065ff07000080fa00000006000000fa0009
:1072a000409920008040eb00014878006099200060
:1072b00081c0b30001487800509920008040eb0065
:1072c000014878000058220001002000804c88000e
:1072d000914c88000080fa00000006000600fa00c9
:1072e000000f780011079800220798001e00780010
:1072f00021072000810f50002100320021072000cb
:10730000810f50000a003c00e20f50001e003200c6
:10731000e20f500003003c00e10f50001300320068
:107320001e003700e30f5000130032001b0037002f
:1073300041072000810f5000090032004107200062
:10734000810f50001200350051072000810f5000be
:1073500011003a00100020003d0007000f00370028
:10736000200020003a0007000c00370057fa070001
:10737000caff070009003700cff9070007003700f0
:107380000000000005003700000000000300370087
:1073900000000000010037000000000010c0b30032
:0873a0000080fa000000060065
:020000040000fa
:1073a800aa090000340000000000000000080000e6
:1073b8001e00000000000000000a0000300000006d
:1073c80000000000100900009a0000000000000002
:1073d8001e0800001200000000000000de09000086
:1073e8000c00000000000000300800000a00000047
:1073f8000000000040080000d0000000000000006d
:107408003a0800000600000000000000000000002c
:020000040000fa
:10741800f03fb1000180b10006003500ee0309001d
:1074280000000000403fb1000180b100fbff3d00bb
:107438001000b000203fb0000200350000800900b5
:08744800000000000000060036
:020000040000fa
:107450000200fa00000f78001e007800e10f5000d3
:1074600002003a00d8fc07000100370000000000cd
:087470000080fa000000060094
:020000040000fa
:020000040005f5
:0457f400ffff0000b3
:020000040000fa
:020000040005f5
:0457f800b6230000d4
:020000040000fa
:020000040005f5
:0457fc006f3e0000fc
:00000001FF
